:100000000C942A000C9447000C9447000C94470071
:100010000C9447000C945C020C9483020C949C0298
:100020000C9447000C9401020C9447000C949D031F
:100030000C9447000C94F4030C9420030C94470098
:100040000C9447000C94990A0C9447000C944700B8
:100050000C94470011241FBECFE5D4E0DEBFCDBF16
:1000600011E0A0E6B0E0EEE5F7E102C005900D92E8
:10007000A435B107D9F714E0A4E5B1E001C01D92A1
:10008000A732B107E1F70E947F000C94AD0B0C94EE
:1000900000008FE187BB8DEF84BB84E081BB82E0F1
:1000A00085BB88E382BB0895F89480E29EE4909338
:1000B0004A028093490240E050E0DA01AA0FBB1FD8
:1000C000FD01E257FE4F8081918188519C4FA75CD2
:1000D000BD4F11969C938E938091490290914A0254
:1000E0002D913C91821B930B90934A02809349027D
:1000F0004F5F5F4F4830510501F778940895CF93D3
:10010000DF938FE187BB8DEF84BB84E081BB82E00E
:1001100085BB88E382BB0E94F2010E941C031092FF
:10012000D70386E48093D80388E08093D90381E0E5
:100130008093DA030E9458031092360289EE92E00F
:1001400090938801809387018BE193E090938A01DB
:1001500080938901789480915B018823E1F3109268
:100160005B010E9422050E9473050E9412060E94F4
:10017000660380E690E00E9479040E9466038FE2A5
:1001800090E09093FA028093F9028EE290E09093CF
:10019000FC028093FB02C0E2DEE4809168018823C8
:1001A00081F181E060E00E94FD04E0918101F0E0D6
:1001B000EE0FFF1FEE0FFF1FE750FC4F808190E016
:1001C0000E948C0583E790E00E94090581E065E0CC
:1001D0000E94FD04E0918101F0E0EE0FFF1FEE0FA1
:1001E000FF1FE950FC4F838190E00E948C0585E75A
:1001F00090E00E94090581E06BE00E94FD041092EE
:10020000680180916901813021F40E94230A0E94D3
:10021000540980916601813071F5809136028130F8
:1002200041F5F894D0934A02C093490240E050E06F
:10023000DA01AA0FBB1FFD01E257FE4F80819181B9
:1002400088519C4FA75CBD4F11969C938E938091D3
:10025000490290914A022D913C91821B930B9093FD
:100260004A02809349024F5F5F4F4830510501F7C2
:1002700078941092660180915E01813021F4109291
:100280005E010E94C50780915D01813011F51092D9
:100290005D01809136028530D1F480915601E09164
:1002A0008101F0E0EE0FFF1FEE0FFF1FE950FC4F42
:1002B000808380916A01813051F4109280010E9404
:1002C0006A0A89E790E00E9479040E9466030E940E
:1002D000C90680915B018130B9F480913602843087
:1002E00089F480915501882331F080915501815026
:1002F0008093550107C084E461E241EE52E022E4BC
:100300000E94EE0810925B0180915A01813009F041
:1003100044CF80913602843009F048C080918E012C
:1003200090918F0180509248880F991F9093E4021A
:100330008093E302809190019091910180509248C6
:10034000880F991F9093E6028093E50280919201B5
:100350009091930180509248880F991F9093EE02DC
:100360008093ED0280919401909195018050924884
:10037000880F991F9093FE028093FD028091960151
:100380009091970180509248880F991F9093000395
:100390008093FF028091980190919901805092483A
:1003A000880F991F90930203809301038091360276
:1003B000853079F49091570180915601981729F072
:1003C0008091560190E00E94AA0580915601809389
:1003D000570110925A01E1CEF89489E189BF7894CF
:1003E0000895089582E083BF1FBC8EBD84EF91E025
:1003F0009BBD8ABD80ED97E099BD88BD81E089BF36
:1004000008951F920F920FB60F9211248F939F930E
:1004100080916E018F5F80936E018150823029F44C
:1004200081E080935E0110926E01809135028F5FB2
:1004300080933502809135028732B9F591E090932F
:100440005C011092350280916D018F5F80936D0188
:1004500080916D01853021F410926D0190935D01C2
:1004600080916B018F5F80936B0180916B0184366B
:1004700039F410926B0181E08093590180935B0104
:1004800080916B01823319F481E080935B0180914C
:100490006C018F5F80936C0180916C018A3029F42C
:1004A00010926C0181E080935A019F918F910F907F
:1004B0000FBE0F901F9018951F920F920FB60F92BC
:1004C00011242F933F934F935F936F937F938F9359
:1004D0009F93AF93BF93EF93FF93E0918701F091C8
:1004E00088010995FF91EF91BF91AF919F918F91F5
:1004F0007F916F915F914F913F912F910F900FBE20
:100500000F901F9018951F920F920FB60F92112403
:100510008F939F939298A99891E090936501809111
:100520005401883011F4909366019F918F910F9040
:100530000FBE0F901F9018951F920F920FB60F923B
:1005400011248F939F93EF93FF93929A1DBC1CBC31
:10055000E0915401F0E0EE0FFF1FE75CFD4F80815A
:10056000918199BD88BD80915401882309F4A99A8D
:1005700080915401823091F0833028F4882341F037
:10058000813099F408C0833061F0843071F40CC07C
:10059000C49AC09A0AC0C098C19A07C0C198C29AAA
:1005A00004C0C298C39A01C0C398809154018F5F60
:1005B0008093540180915401893010F010925401BD
:1005C000FF91EF919F918F910F900FBE0F901F9011
:1005D000189580916F0190917001892B81F486B5F7
:1005E00097B590937601809375018EB58F7B8EBD04
:1005F00081E090E09093700180936F01089586B53B
:1006000097B590937401809373012EB520642EBD2D
:100610002091750130917601821B930B90937201AA
:10062000809371011092700110926F0190934003BA
:1006300080933F030895089517B88FEE86B9089503
:100640001F920F920FB60F9211248F939F93EF93E7
:10065000FF9316B8E0915801F0E084B195B1EE0F28
:10066000FF1FE257FE4F91838083809158018F5F77
:100670008093580180915801873010F010925801F2
:100680008091580187B98FEE86B980918E01909143
:100690008F01969587959695879580935601FF9142
:1006A000EF919F918F910F900FBE0F901F90189513
:1006B00080E189B910BC88E18AB986E880BD82EC06
:1006C0008BB908955D9BFECF8CB908958091DE00B3
:1006D0005D9BFECF8CB98091DF005D9BFECF8CB916
:1006E000089527E030E061E070E0482F50E0F0E34B
:1006F000E1E3CB01022E02C0880F991F0A94E2F7B2
:10070000842395231816190624F45D9BFECFECB9BB
:1007100003C05D9BFECFFCB9215030408FEF2F3FCF
:10072000380739F78091DE005D9BFECF8CB9809150
:10073000DF005D9BFECF8CB908951F920F920FB61C
:100740000F9211248F939F93EF93FF939CB19093FB
:10075000EC039D3099F480917801813079F4109206
:10076000780180936901E0912303F0E0E55BFD4FA0
:10077000908380912303809377012DC0809178012D
:10078000882319F0813039F514C0933241F48091F7
:100790006901882321F481E080937801979A10926F
:1007A000230380912303E82FF0E0E55BFD4F908366
:1007B0000CC0E0912303F0E0E55BFD4F9083809156
:1007C0002303853930F4809123038F5F80932303C3
:1007D00002C010927801FF91EF919F918F910F903D
:1007E0000FBE0F901F9018951F920F920FB60F9289
:1007F00011242F933F934F935F936F937F938F9326
:100800009F93AF93BF93EF93FF9380913602843011
:1008100019F58091E0008823D9F4809179019091B5
:100820007A01019690937A0180937901FC01EF5B44
:10083000FC4FE081ED3019F08639910539F41092C2
:100840007A011092790181E08093E000ECB904C054
:1008500010927A0110927901809136028330C1F5AD
:1008600080916701813081F08230C9F0882381F561
:1008700010BC85E089B91CB80E9401080E941C08C0
:1008800081E08093670124C010BC89B91CB882E064
:10089000809367011092A1011092A00119C08AE112
:1008A0008A95F1F78091A0019091A101FC01EA5491
:1008B000FE4F20812CB901969093A1018093A00155
:1008C0008091A0019091A101C29711F4109267014B
:1008D000FF91EF91BF91AF919F918F917F916F9118
:1008E0005F914F913F912F910F900FBE0F901F90EE
:1008F0001895DC010D900020E9F71197A81BB90BA2
:1009000020E030E0FC01E20FF31FE0815D9BFECFB1
:10091000ECB92F5F3F4FA217B307A0F708950F93CD
:100920001F93DF93CF93CDB7DEB764970FB6F894DC
:10093000DEBF0FBECDBF8E010F5F1F4FB8014AE073
:1009400050E00E94680BC8010E94790464960FB6BB
:10095000F894DEBF0FBECDBFCF91DF911F910F91F5
:10096000089580FF02C0AC9A01C0AC9881FF02C01C
:10097000AD9A01C0AD9882FF02C0AE9A01C0AE9898
:1009800083FF02C0AF9A0895AF980895AA9A80E1B4
:1009900097E20197F1F7AA980895FF920F931F939A
:1009A000F82E82958F700E94B104AA9A00E117E296
:1009B000C8010197F1F7AA988F2D0E94B104AA9A55
:1009C000C8010197F1F7AA981F910F91FF90089520
:1009D000AB9A0E94CD040895AB980E94CD04AB9AC7
:1009E000089581E00E94EC0408958CE00E94EC04DC
:1009F00008958DE00E94EC040895882319F4862F51
:100A0000805804C0813011F4862F80540E94EC0479
:100A100008950F931F93CF93DF93FC010190002063
:100A2000E9F731970E2F081BEC0110E004C0899103
:100A30000E94E8041F5F1017D0F3DF91CF911F9140
:100A40000F910895EF92FF920F931F9300E117E229
:100A5000C8010197F1F7AB9883E00E94B104AA9A0C
:100A6000C8010197F1F7AA9880E2E82E8EE4F82EEB
:100A7000C7010197F1F783E00E94B104AA9AC80167
:100A80000197F1F7AA98C7010197F1F783E00E9457
:100A9000B104AA9AC8010197F1F7AA9882E00E94CE
:100AA000B104AA9AC8010197F1F7AA98C701019762
:100AB000F1F788E20E94EC048EE00E94EC0481E0F1
:100AC0000E94EC0481EE90E00E94090581E06AE05A
:100AD0000E94FD0486EE90E00E9409051F910F918F
:100AE000FF90EF9008950E94F10480E063E00E947F
:100AF000FD048BEE90E00E94090581E062E00E9417
:100B0000FD0486EF90E00E9409050E94F504859996
:100B1000FECF0E94F10408950F931F93DF93CF93AC
:100B200000D000D00F92CDB7DEB78E010F5F1F4F00
:100B3000B8014AE050E00E94680BC8010E94090514
:100B40000F900F900F900F900F90CF91DF911F910A
:100B50000F9108951F93182F0E94F50480E067E01D
:100B60000E94FD0483E091E00E94090580E067E0B7
:100B70000E94FD04812F90E00E948C050E94F904E0
:100B800080916401813039F0823039F0882349F452
:100B900080E060E004C080E001C081E06BE00E9482
:100BA000FD041F91089580916A01882349F481E032
:100BB00080936A016BE00E94FD0487E091E012C01F
:100BC00010926A01E0918101F0E0EE0FFF1FEE0F3D
:100BD000FF1FE950FC4F108281E06BE00E94FD0492
:100BE0008DE091E00E94090581E06BE00E94FD0428
:100BF000089580916A018823A1F4109236028AE058
:100C00008093620110925F0180E062E00E94FD0427
:100C1000809181018F5C0E94E80480E062E00E9484
:100C2000FD04089581E080936201109263011092A7
:100C300036020E94F10480E060E00E94FD0483E13E
:100C400091E00E94090580E069E00E94FD048BE1CB
:100C500091E00E94090581E060E00E94FD0482E2CB
:100C600091E00E94090581E069E00E94FD048AE2AA
:100C700091E00E9409050E94F90480E060E00E9472
:100C8000FD0410925F01089585E0809362010E9447
:100C9000F10481E069E00E94FD0480E391E00E949C
:100CA00009050E94F90481E069E00E94FD041092A8
:100CB0005F010E94F5040E948E08089584E08093ED
:100CC00062010E94F10481E069E00E94FD0480E37A
:100CD00091E00E9409050E94F90481E069E00E9408
:100CE000FD0410925F010E94F5040E94E60708953A
:100CF00086E0809362010E94F10481E069E00E9435
:100D0000FD0480E391E00E9409050E94F90481E05E
:100D100069E00E94FD0410925F010E94F5040E94A8
:100D2000A808089587E080936201109263010E94F1
:100D3000F10480E060E00E94FD0485E391E00E9400
:100D40000905809181018F5C0E94E80480E064E0E5
:100D50000E94FD0488E391E00E94090580E06BE0B9
:100D60000E94FD0480E391E00E94090581E06BE0B0
:100D70000E94FD048DE091E00E9409050E94F904A3
:100D800080E060E00E94FD0410925F010E94600A12
:100D9000089580915F01882309F48AC080916201DF
:100DA000813099F580915F01181624F480916301D8
:100DB0008F5F03C0809163018150809363018091B4
:100DC000630187FF03C083E0809363018091630127
:100DD000843014F01092630180916301813061F0DE
:100DE00082301CF4882331F010C0823039F0833017
:100DF00061F407C080E003C080E004C081E060E0EF
:100E000002C081E069E00E94FD04809162018730A8
:100E100079F580915F01181624F4809163018F5F4A
:100E200003C08091630181508093630180916301CD
:100E300087FF03C082E08093630180916301833068
:100E400014F010926301809163018093640180919A
:100E50006301813039F0823039F0882349F480E031
:100E600060E004C080E001C081E06BE00E94FD040E
:100E7000809162018A30D1F480915F01909181016B
:100E8000181614F49F5F01C09150909381018091D6
:100E90008101893010F010928101809181018F5C75
:100EA0000E94E80480E062E00E94FD0410925F016D
:100EB000859909C080918D01813051F410928D0087
:100EC00010928D0105C081E080938D0180938D008B
:100ED00080918D00882309F057C080916201853090
:100EE00049F1863034F4813061F0843009F049C032
:100EF0001EC0873039F1873014F18A3009F041C0C3
:100F000034C080916301823011F40E945E068091AA
:100F10006301882311F40E944406809163018330A9
:100F200011F40E94920681E080938D002AC00E94F5
:100F3000F60702C00E94A1080E94120622C00E9469
:100F4000B508FACF80916301882311F40E94F90556
:100F500080916301813011F40E9412068091630137
:100F6000823079F40E94D3050CC087E0809362013F
:100F70001092630180E060E00E94FD0485E08093B0
:100F8000360281E080938D000895F89480B390E05C
:100F900024E0969587952A95E1F7982F9170839B89
:100FA00002C083E09827789480918C00981B90FF72
:100FB0000CC080918C00890F80938C0080915F0120
:100FC00081509270890F80935F01089583E0809330
:100FD0003602F89410BC81E089B98EE880BD88E4BF
:100FE0008AB978941CB8109267010895109236025D
:100FF000F89410BC81E089B98EE880BD1AB8789465
:10100000089520E030E040E012C0F901EE0FFF1F2C
:10101000E257FE4F808191819695879596958795A9
:10102000F901EA54FE4F80832F5F3F4F4F5F4630F8
:1010300064F34093ED0308951F93CF93DF931092D1
:10104000ED03C0EFD3E013E060C0FF27E7FDF095AC
:10105000EA54FE4F80818093EE031092EF0390E0FC
:1010600060EF73E04AE050E00E94680BFE010190DF
:101070000020E9F73197E05FF340E093F5038091BA
:10108000ED03682F772767FD70958430B4F4660F01
:10109000771F660F771F80E00E94FD048EE391E0CA
:1010A0000E9409058091F503912F981B6091ED0333
:1010B000660F660F690F80E01DC064507040660FB8
:1010C000771F660F771F81E00E94FD048EE391E099
:1010D0000E9409058091F503612F681B8091ED0343
:1010E000992787FD90950497880F991F880F991F5E
:1010F000680F81E00E94FD0480EF93E00E940905E3
:101100008091ED038F5F8093ED03E091ED03E63076
:101110000CF49BCFDF91CF911F910895F89481E05B
:10112000809336021FBC82E08EBD84EF91E09BBDB0
:101130008ABD80ED97E099BD88BD89E189BF78942B
:101140000895F8941092360281E089BF789408954A
:1011500084E08093360280E189B910BC88ED8AB9B9
:1011600086E880BD82EC8BB908951092360280E14A
:1011700089B910BC1AB886E880BD82EC8BB9089595
:10118000DC0120E030E040E050E008C0FA01EF5B15
:10119000FC4F8081280F311D4F5F5F4F4A175B075F
:1011A000A8F33F70C90136E0969587953A95E1F727
:1011B000835CFD01EF5BFC4F808311962F73235CF2
:1011C000FD01EF5BFC4F2083AE5BBC4F8DE08C9349
:1011D0001092E000809141038CB90895CF93DF9382
:1011E000EA01B22F93E2909341036093420380930C
:1011F000430363E070E0A0E04EC0FE01EA0FF11D82
:101200009081AF5FB15019F430E040E00FC0FE01B3
:10121000EA0FF11D4081AF5FB15011F430E006C01C
:10122000FE01EA0FF11D3081AF5FB150892F869525
:101230008695835CFB01EF5BFC4F8083242F229516
:101240002F70892F90E08370907054E0880F991F61
:101250005A95E1F7282B235CFB01EE5BFC4F2083C2
:10126000842F90E08F709070880F991F880F991FBE
:10127000232F2295269526952370282B235CFB018E
:10128000ED5BFC4F20833F73335CFB01EC5BFC4F59
:1012900030836C5F7F4FBB2309F0AFCFCB010E943F
:1012A000C008DF91CF910895DF93CF93CDB7DEB71C
:1012B00060970FB6F894DEBF0FBECDBF8091E000FF
:1012C000882309F45FC06091F6036F3F59F0605DB9
:1012D00081E4AE014F5F5F4F20E10E94EE088FEF87
:1012E0008093F60380917B01813061F487E461E0B3
:1012F00041EE53E02BE00E94EE0810927B0182E069
:101300008093550180917C01813061F482E080936B
:10131000550186E561E047ED53E02AE00E94EE08C2
:1013200010927C0180917D018130E1F482E0809314
:10133000550180917F0144E1849FA001112442570F
:101340005F4F805D60E024E10E94EE0880917F01A4
:101350008F5F80937F018150843011F410927F0160
:1013600010927D0180917E01813061F482E0809352
:10137000550184E461E241EE52E022E40E94EE086D
:1013800010927E0160960FB6F894DEBF0FBECDBFFF
:10139000CF91DF9108951F93CF93DF93EC0170E01D
:1013A000A22FB0E0119748C0E42FF0E0E55BFD4FBD
:1013B00030814F5FE42FF0E0E55BFD4F50814F5FE0
:1013C000E42FF0E0E55BFD4F10814F5FE42FF0E08C
:1013D000E55BFD4F20814F5F842F90E08A179B07CC
:1013E00074F55D53FE01E70FF11D852F82958F7017
:1013F0003D53330F330F382B3083613001F1912F80
:101400009D537F5FFE01E70FF11D71505295507F94
:10141000892F86958695582B5083623081F06350D2
:101420007E5FFE01E70FF11D9295990F990F907C59
:101430002D53922B90837F5F662309F0B5CFDF9108
:10144000CF911F910895DF93CF9300D000D0CDB7F7
:10145000DEB780914D028736C1F0883628F4813698
:1014600041F0833621F51DC08836B9F08637F9F48E
:1014700010C020917701CE01019664E043E00E9404
:10148000CB0989818093F60312C081E080937B01B0
:101490000EC081E080937C010AC081E080937D01D1
:1014A00006C081E080937E0182E080935501109216
:1014B00069010F900F900F900F90CF91DF910895D9
:1014C00085E08093360211B88CE080B908951092BF
:1014D0003602089585EA86BF089584E986BF089597
:1014E00084E986BF1092800183B11092810180E867
:1014F00086BF12B813B811B810B885E080933602D1
:1015000011B88CE080B985EA86BF11B813B885E8B8
:1015100086BF089511B883B985E886BF089583B959
:1015200085E886BF089585EC86BF089585E886BF67
:1015300008951F920F920FB60F9211242F933F938D
:101540004F935F936F937F938F939F93AF93BF93CB
:10155000EF93FF9381E491E00E9479040E94660377
:10156000809180018F5F809380018150833009F4E6
:101570004EC0843028F48130A9F0823010F50AC0C2
:10158000853009F470C0853008F446C0863009F013
:1015900089C075C011B88091810190E08996880F4B
:1015A000991F0BC0E0918101F0E0EE0FFF1FEE0FDD
:1015B000FF1FE950FC4F808111B883B985E886BFD1
:1015C00073C081B18033C9F480918601882321F4EE
:1015D000809181018093860180918101E82FF0E064
:1015E000EE0FFF1FEE0FFF1FED50FC4F9181892F73
:1015F0008F778F3711F09F5F918384E986BF8AE0F0
:1016000090E0909338028093370285EAD8CF80919A
:101610008101880F8D5AD0CF81B1E0918101803452
:1016200079F0F0E0EE0FFF1FEE0FFF1FE950FC4FC7
:1016300081818F77818384E986BF109280010CC0FD
:10164000F0E0EE0FFF1FEE0FFF1FE950FC4F81810E
:101650008068818385EC86BF8091860180938301B9
:101660001092860121C083B1E0918101F0E0EE0F7C
:10167000FF1FEE0FFF1FE750FC4F80839FCF83B10A
:10168000E0918101F0E0EE0FFF1FEE0FFF1FE95028
:10169000FC4F838384E986BF1092800181E08093B0
:1016A000680102C01092800186B7806886BFFF91F2
:1016B000EF91BF91AF919F918F917F916F915F91CA
:1016C0004F913F912F910F900FBE0F901F90189543
:1016D000FB019F01E8944230C4F04532B4F44A3033
:1016E00029F497FB1EF4909581959F4F642F7727DF
:1016F0000E94990B805D8A330CF0895D8193CB0148
:101700000097A1F716F45DE251931082C9010C9481
:10171000890BDC01FC01672F71917723E1F7329788
:1017200004C07C916D9370836291AE17BF07C8F3BC
:101730000895AA1BBB1B51E107C0AA1FBB1FA61718
:10174000B70710F0A61BB70B881F991F5A95A9F76A
:0E17500080959095BC01CD010895F894FFCFCF
:10175E00736572766F7465737420562E20302E3733
:10176E002E7300410050574D006932635F737461F0
:10177E007274004B2000000000003D0001013D3D51
:10178E003D204D6963726F636F62746572203D3DDB
:10179E003D0046432D53696D756C61746F72205612
:1017AE0020302E31200020202020204550492D545D
:1017BE0045414D20202020202000202020202020C8
:1017CE00776F7769652020202020202020000D0AC9
:1017DE00016875687500416B6B75004550492D5455
:1017EE0065737465720056657273696F6E20302E64
:1017FE003264002020200053746F702000537461F7
:10180E0072740050504D2D4F75740050504D2D492F
:10181E006E00444D582D4F757400424C432D5400AC
:10182E004578697400413D00533D20203000202052
:10183E000054574920566563746F72207265616358
:04184E006865640065
:00000001FF
